:100000000C9464000C9481000C9481000C94810089
:100010000C9481000C9481000C9481000C9481005C
:100020000C9481000C9481000C9481000C940104C8
:100030000C942B040C9481000C9481000C9481008E
:100040000C9481000C9481000C9481000C9481002C
:100050000C9481004F4B004552524F52002B434DA0
:1000600047523A002B434C49503A002B4350494EDB
:100070003A0052494E47002B434C43433A00540048
:1000800057005D0064006B007200770053494D20FB
:1000900050554B0053494D2050494E0041542B437D
:1000A0004855500D0041542B434C43430D000D0067
:1000B00041542B4350494E3D0041542B4350494E2F
:1000C0003F0D0041540D000011241FBECFE5D4E0C8
:1000D000DEBFCDBF10E0A0E6B0E0E8E4FAE002C089
:1000E00005900D92AE36B107D9F711E0AEE6B0E05B
:1000F00001C01D92AA3EB107E1F70E94B0030C9423
:1001000022050C9400008091220190912301A0917E
:100110002401B091250180618093220190932301F5
:10012000A0932401B093250108958091220190911C
:100130002301A0912401B0912501886080932201C0
:1001400090932301A0932401B0932501089508956D
:1001500008958091220190912301A0912401B091F2
:10016000250190618093220190932301A0932401A3
:10017000B09325010895CF93DF939C018091DD0119
:10018000882309F443C0C90162E270E00E940705B8
:10019000FC010097D9F1DC01119681818B3209F4C1
:1001A0001196ED0140E050E0642FE42FE695F0E079
:1001B000E452FE4F968140FD02C080EF01C08FE007
:1001C00040FD03C024E030E002C020E030E089239D
:1001D00090E002C0959587952A95E2F7782F282F11
:1001E00030E0205D3F4F888190E02817390739F4CF
:1001F0006F5F4F5F5F4F219641315105A9F67A300D
:1002000088F0A60FB11D8C91823261F48091DC01DF
:1002100087FF05C08BB390E489278BBB03C08F5F3A
:1002200080936F00DF91CF910895CF93DF93EC011E
:1002300064E970E00E94ED04892B51F08091220165
:1002400090912301A0912401B0912501806210C0FA
:10025000CE016CE870E00E94ED04892B89F080915A
:10026000220190912301A0912401B0912501806485
:100270008093220190932301A0932401B093250140
:10028000DF91CF910895FF920F931F93CF93DF9348
:100290003FC080916E00C82FD0E00E946504C25418
:1002A000DF4F888380916E00E82FF0E0E254FF4F2B
:1002B000E081EA3069F1ED3041F5882319F1CEE7AC
:1002C000D0E0FF24FE0105911491C8010E94D604DC
:1002D000AC018EEB90E0B8010E94DF04892B69F439
:1002E000EF2DF0E0EE0FFF1FE05AFF4F0190F0817D
:1002F000E02D8EEB90E0099505C0F394229687E0FF
:10030000F81601F710926E0003C08F5F80936E00A5
:100310000E94A204892B09F0BCCFDF91CF911F91DD
:100320000F91FF900895FC01E056FF4F83E6819303
:1003300082E0819388E0819388E2819388E68193CB
:1003400084EF8083089520E030E0622FE22FE6956D
:10035000F0E0E452FE4F928120FD02C080EF01C028
:100360008FE020FD03C044E050E002C040E050E0D8
:10037000892390E002C0959587954A95E2F78A30E7
:1003800030F46F5F2F5F3F4F28303105F1F6643056
:1003900010F482E0089520E030E0622FE22FE6952D
:1003A000F0E0E452FE4F968120FD02C080EF01C0D4
:1003B0008FE020FD03C044E050E002C040E050E088
:1003C000892390E002C0959587954A95E2F78A3097
:1003D00030F46F5F2F5F3F4F20313105F1F664300D
:1003E00010F080E0089583E008952091740030912A
:1003F00075002F5F3F4F309375002093740097E096
:10040000203D390710F4DF980895823079F0833069
:1004100020F4813009F03BC005C0833059F08430AE
:10042000B1F51FC0245C394070F007C0285B3B4029
:1004300050F003C02C5A3D4030F081E090E09093A2
:1004400075008093740080917400909175006AEF3C
:1004500070E00E94AF04892BD1F48BB380588BBB22
:100460000895205A3F4030F081E090E0909375006D
:100470008093740080917400909175006AEF70E031
:100480000E94AF04892B19F48BB380588BBB08955D
:100490008091DC0187FD1FC020916F002223B1F005
:1004A00080917200909173000196909373008093F5
:1004B000720001978053954738F0109273001092A4
:1004C0007200215020936F00DE9A089510927300FD
:1004D00010927200DE980895CF93DF938091780098
:1004E000833009F471C0843030F48130D9F0823027
:1004F00008F05DC00AC0853009F4F2C0853008F408
:10050000BFC0863009F027C10FC183EC90E00E9484
:100510009404809178008093770081E08093780044
:1005200082E0FBC08091220190912301A0912401DF
:10053000B091250184FF15C08F7EA070B0708093AC
:10054000220190932301A0932401B093250180916F
:1005500076008093780080912601813011F410920A
:1005600026018091220190912301A0912401B09154
:10057000250183FF12C0877FA070B0708093220195
:1005800090932301A0932401B093250180917700DB
:10059000833019F484E0809326018091700090915B
:1005A00071008D5D954008F4D8C081E066C089EB8C
:1005B00090E00E949404809178008093770081E01D
:1005C0008093780083E0A9C080912201909123015B
:1005D000A0912401B091250185FF41C08F7DA070BD
:1005E000B0708093220190932301A0932401B093D3
:1005F000250180EB90E00E949404C0E0D0E0CE01A1
:100600008695E82FF0E0E452FE4F9281C0FD02C0D3
:1006100080EF01C08FE0C0FD03C024E030E002C0E5
:1006200020E030E0892390E002C0959587952A95D7
:10063000E2F78A3038F4805D0E9482042196C83047
:10064000D105E9F68EEA90E00E949404809178004A
:100650008093770081E08093780084E05EC086FF1D
:1006600076C08F7BA070B07080932201909323019D
:10067000A0932401B093250184E0809326016BC0F0
:100680008091220190912301A0912401B091250134
:1006900094FF1DC09F7EA070B07080932201909344
:1006A0002301A0932401B093250185EA90E00E94E4
:1006B0009404809178008093770081E080937800A3
:1006C00085E0809376001092710010927000809106
:1006D000700090917100815A9F4008F43EC03BC069
:1006E000209170003091710087E0203D3807A8F11B
:1006F0008091DC0187FF05C0DE9903C0205137429D
:1007000060F18CE990E00E949404809178008093DD
:10071000770081E08093780086E0809376001092E5
:1007200071001092700019C08091220190912301F4
:10073000A0912401B09125019F7EA070B07080939C
:10074000220190932301A0932401B093250184E01A
:100750008093780002C010927800DF91CF910895C5
:100760002BE088E190E00FB6F894A89581BD0FBE0C
:1007700021BD90E89ABBD69A82E081BB98B9DF98F8
:10078000DE9883E083BF83E390E00E94500487E219
:1007900091E00E9493018CED91E060E070E04EE00A
:1007A00050E00E9412058CED91E00E94A30180931D
:1007B000260112BE789482B78E37F8F012BE80916F
:1007C0007000909171000196909371008093700079
:1007D00001972FEF8F3F920721F490937100809340
:1007E000700080912601823010F40E946C020E94F9
:1007F0004802809126010E94F5010E944301A895BC
:10080000DACF1F920F920FB60F9211242F938F936E
:100810009F93EF93FF939BB12CB1E091BB00EF5FEF
:10082000EF718091BC00E81711F482E008C0892FB5
:100830008871E093BB00F0E0E756FF4F2083809380
:10084000BD00FF91EF919F918F912F910F900FBE5F
:100850000F901F9018951F920F920FB60F921124B0
:100860008F939F93EF93FF939091B9008091BA007B
:10087000981761F0E091BA00EF5FEF71E093BA0072
:10088000F0E0E758FF4F80818CB901C05598FF9187
:10089000EF919F918F910F900FBE0F901F90189521
:1008A0009C011092B9001092BA001092BB001092F5
:1008B000BC0097FF03C082E08BB93F7730BD29B9F8
:1008C00088E98AB986E880BD08959091BB0080913F
:1008D000BC00981719F420E031E012C0E091BC0090
:1008E000EF5FEF71E093BC00F0E0E756FF4F30811F
:1008F0002091BD00922F80E0AC01430F511D9A0161
:10090000C9010895282F9091B9009F5F9F71809130
:10091000BA009817E1F3E92FF0E0E758FF4F208382
:100920009093B900559A0895CF93DF93EC0102C0DC
:100930000E948204FE01219684918823C9F7DF91E9
:10094000CF9108958091BB002091BC0090E04F961C
:10095000821B91096FE170E00E94C3040895AA1BF5
:10096000BB1B51E107C0AA1FBB1FA617B70710F09A
:10097000A61BB70B881F991F5A95A9F780959095CC
:10098000BC01CD01089597FB092E07260AD077FDFB
:1009900004D0E5DF06D000201AF4709561957F4FF2
:1009A0000895F6F7909581959F4F0895FC01059065
:1009B0000020E9F7809590958E0F9F1F0895FB0109
:1009C000DC014150504030F08D910590801919F4B0
:1009D0000020B9F7881B990B0895FB015591552309
:1009E000A9F0BF01DC014D9145174111E1F759F420
:1009F000CD010590002049F04D9140154111C9F3FA
:100A0000FB014111EFCF81E090E001970895FC01D7
:100A10008191861721F08823D9F799270895319776
:100A2000CF010895DC01CB01FC01E199FECF06C0A6
:100A3000FFBBEEBBE09A31960DB20D924150504093
:080A4000B8F70895F894FFCF08
:0E0A480083009500A700A8001501A900BB00BF
:00000001FF
